:100000000C948B000C94DA000C94BF000C94BF008D
:100010000C94BF000C94BF000C94BF000C94BF0064
:100020000C94BF000C94BF000C94BF000C94BF0054
:100030000C94BF000C94BF000C94BF000C94BF0044
:100040000C94C90E0C94BF000C9442120C946F12C5
:100050000C94BF000C94BF000C94BF000C943E0E97
:100060000C94BF000C94BF000000000800020100C7
:100070000003040700000000000000000102040863
:100080001020408001020408102001020408102002
:10009000040404040404040402020202020203032E
:1000A00003030303000000002300260029000000D2
:1000B0000000250028002B0000000000240027007D
:1000C0002A000902120001010080FA090400000060
:1000D0000000000012011001FF000008C016DC053E
:1000E00000010102000116034C00450044004300DA
:1000F0006F006E00740072006F006C0012036F00DE
:1001000062006400650076002E0061007400040344
:100110000904810E951211241FBECFEFD8E0DEBF77
:10012000CDBF14BE0FB6F894A89580916000886189
:1001300080936000109260000FBE12E0A0E0B1E07A
:10014000E6E3F4E302C005900D92A031B107D9F7C0
:1001500024E0A0E1B2E001C01D92AE35B207E1F7A4
:1001600010E0CBE8D0E004C02197FE010E94C9193D
:10017000C938D107C9F70E9464090C944D190C9431
:100180000000A82FB92F80E090E041E050EA609590
:1001900030E009C02D9182279795879510F084272C
:1001A0009527305EC8F36F5FA8F30895EADF8D935B
:1001B0009D930895CF93CFB7CF93C3954C9BE9F709
:1001C0004C9B09C04C9B07C04C9B05C04C9B03C07B
:1001D0004C9B01C0A1C0DF93C0914704DD27C85BE1
:1001E000DB4F4C9B02C0DF91EBCF2F930F931F93FC
:1001F00009B12FEF04FB20F94F933F9319B14FEF53
:10020000012704FB21F93BE031C04E7F012F19B1DA
:10021000216028C0102F4D7F2260000009B129C045
:100220004B7F2460012F000019B12BC019B1477F0B
:1002300028602AC04F7E09B120612CC04F7D19B1C2
:1002400020622FC04F7B09B1206432C0422709B120
:1002500049934FEF0000102714FB20F919B11471D6
:10026000C9F1297F91F2012704FB21F909B1237F0C
:1002700089F2315058F1102714FB22F919B1277E69
:1002800079F2012704FB23F92F7C81F209B11027B1
:1002900014FB24F92F7971F200C019B1012704FB76
:1002A00025F92F7359F200C009B1102714FB26F964
:1002B000223040F200C019B1012704FB27F9243095
:1002C00028F64F77206819B10000F9CF11E01CBB68
:1002D000002717C03B503195C31BD04011E01CBB19
:1002E0000881033CE9F00B34D9F0209146041981D0
:1002F000110F1213EDCF093641F10D3211F0013E0D
:1003000039F7009342043F914F911F910F912F9124
:10031000DF91CCB3C0FD51CFCF91CFBFCF91189516
:1003200020914204222379F310914304112311F503
:10033000343012F130934304209341041091470468
:100340003BE0311B3093470417C000914304013058
:100350008CF40AE530910C0134FD10C000930C01BF
:10036000C6E3D4E00FC02795A8F45150A9F4220F9A
:100370000000F9CF4AE503C042ED01C0432FC4E1BC
:10038000D0E032E01AB114615C9A1AB90BB120E4E2
:1003900014E15F93012756E00BB9279520F45150E3
:1003A00021F4220FF9CF012756E000003B5A0BB988
:1003B000D0F2279528F4515029F4220F0000F9CFEC
:1003C000012756E027950BB920F4515021F4220F54
:1003D000F9CF012756E0299133230BB921F60B7E83
:1003E00010914504110FC651D0400BB911F0109374
:1003F000460411E01CBB00611AB11B7E402F4B7EEE
:100400005F9100C000C00BB91AB94BB97CCFFC0199
:1004100081E090E09383828382E390E09183808304
:100420001582148281E086831186138612861086D7
:1004300017820895AF92BF92CF92DF92EF92FF9210
:100440000F931F93CF93DF93D82EEB018A016DE0BA
:1004500071E086E993E00E9413136CE271E086E993
:1004600093E00E9406134AE050E06D2D86E993E088
:100470000E9419148FEF7801C12CD81215C0CE013B
:100480000E94070280E0DF91CF911F910F91FF90B2
:10049000EF90DF90CF90BF90AF9008957801E80E75
:1004A000F91E0E946118C394C7010E94E919B82E71
:1004B000C70101960E94E9199B2DDC10EFCF045073
:1004C00011090E191F09080F191F16950795169582
:1004D00007951B830A830E946118C70102960E9438
:1004E000E9198E83C70103960E94E919182FC701E5
:1004F00004960E94E919912F998388830E946118BC
:1005000018861F82C70105960E94E9198987C701CD
:1005100006960E94E9198A876701E8E0CE0ED11C91
:10052000C70107960E94E9198B870E9461188E0106
:10053000EE24E394F12C0B5F1F4F8A819B81E81618
:10054000F90618F01D821C829DCFF801A280B380AD
:10055000C6010E94E919A80EB11CF801B086A78255
:10056000C60101960E94E919F80181870E9461186D
:10057000C60102960E94E919F80182875601F4E04B
:10058000AF0EB11CC60103960E94E919F8018387DA
:100590000E946118FFEFEF1AFF0A6501CCCF3F926E
:1005A0004F925F926F927F928F929F92AF92BF9283
:1005B000CF92DF92EF92FF920F931F93CF93DF932F
:1005C000EC0180E090E00E94E919182F81E090E0B2
:1005D0000E94E919912F9983888382E090E00E941C
:1005E000E919182F83E090E00E94E919912F9B836D
:1005F0008A8384E090E00E94E919782E8C8385E05C
:1006000090E00E94E919682E8D837E0128E9E20EB0
:10061000F11C512C06E010E0561031C06E0178013B
:10062000912CF4E0CF0ED11C971088C0FE01EC563F
:10063000FF4F81E090E0819391938FEF81938083CE
:1006400082E28E831F82198618861B861A8624E012
:10065000929EC0011124800F911FDF91CF911F91B5
:100660000F91FF90EF90DF90CF90BF90AF909F9051
:100670008F907F906F905F904F903F900895C8014A
:100680000E94E919D82EC80101960E94E91990E04C
:10069000A0E0B0E05C0199248824BD28C80102963E
:1006A0000E94E919D82EC80103960E94E919882AE8
:1006B0009D28F70180829182A282B3825801F5E0E1
:1006C000AF0EB11CC80104960E94E919382EF7013B
:1006D00084836701F5E0CF0ED11C8501412C4310C6
:1006E0000BC024E0429E800111240A0D1B1D53946F
:1006F00089E1E80EF11C90CFC8010E94E919982EFB
:10070000C80101960E94E919992DF6019183808311
:10071000C80102960E94E919F60182834801F4E0BB
:100720008F0E911CC80103960E94E919F60183837C
:100730004394F4E0CF0ED11C8401D1CFC7010E94B5
:10074000E919B82EC70101960E94E9199B2DF601FF
:1007500091878087C70102960E94E919F601828776
:100760005701F4E0AF0EB11CC70103960E94E919CE
:10077000F60183879394750154CF2F923F924F9245
:100780005F926F927F928F929F92AF92BF92CF9221
:10079000DF92EF92FF920F931F93CF93DF9300D0DE
:1007A00000D0CDB7DEB78B839C837B01AB81BC814E
:1007B0008D919C911197892B09F0DCC012968D9137
:1007C0009C91892B09F0D6C0CB010E9422164B01C7
:1007D0005C01B501A401C7010E9474168C01EB8174
:1007E000FC81828593858017910708F59801281B65
:1007F000390BC901EB81FC81208531858217930774
:1008000008F49EC03580E856FF4F20E040E050E0FD
:10081000BA01C12CD12C321211C0EB81FC81848130
:1008200090E040E050E0BA0120E030E06DC0D80137
:10083000A81BB90BCD01805A984DDCCF4080518068
:1008400062807380481459046A047B0450F4348134
:10085000CF0105969A838983B301A201212C32111D
:1008600024C080E02F5F79968115A9F2C7010E940C
:100870007416AC0124E0C29EF001112439E1D39E2C
:10088000E00DF11D11248B819C81E80FF91FE356C7
:10089000FF4F80819181AB81BC8119969C938E938F
:1008A000189714969C919D0D45C0A981BA814D90D1
:1008B0005C90DB01CA01840D951DA11DB11D2C01A9
:1008C0003D0188169906AA06BB0648F0A981BA819F
:1008D0001496BA83A9832394B301A201C0CFC22C7A
:1008E000D22E81E0BFCFA485B5854A015B018A0E77
:1008F0009B1EA11CB11C081519052A053B0538F0E3
:1009000034969F5FB501A4018913EDCF9D2DE92F8A
:10091000F0E03396EE0FFF1FEE0FFF1F2B813C819F
:10092000E20FF31F20813181AB81BC8119963C938A
:100930002E931897EB81FC819683C7825387428759
:10094000EB81FC8186810F900F900F900F90DF91CB
:10095000CF911F910F91FF90EF90DF90CF90BF90BC
:10096000AF909F908F907F906F905F904F903F904F
:100970002F900895C7010E94B11660EA75E00E94A9
:1009800060199C01AB81BC8112968D919C9113974B
:100990004D915C912417350718F02817390738F066
:1009A00022E2EB81FC81268393878287C9CFAB81CA
:1009B000BC811A968D919C911B97A901481B590BDC
:1009C00018968D919C9119974817590708F4B8CF3C
:1009D00016968C9116978232F9F090E00196149653
:1009E0006C9170E00E947419482FEB81FC81468362
:1009F00033872287FC013396EE0FFF1FEE0FFF1F98
:100A00002B813C81E20FF31F80819181D9011996DE
:100A10009C938E93189794CF40E080E090E0E5CFD0
:100A200088E198E00FB6F894A895809360000FBE17
:100A300090936000FFCFCF92DF92EF92FF920F93DF
:100A40001F93CF93DF93EC0119811A3180F4E12FCA
:100A5000F0E0EF5FF54E0C94C9190E941A0F6093F5
:100A60001A0270931B0280931C0290931D0210E0E7
:100A7000812FDF91CF911F910F91FF90EF90DF9029
:100A8000CF9008950E941A0F609316027093170278
:100A90008093180290931902EACF809116029091E8
:100AA0001702A0911802B091190240911A025091B8
:100AB0001B0260911C0270911D02841B950BA60BFA
:100AC000B70B8093120290931302A0931402B09379
:100AD000150282E192E0909335048093340414E08F
:100AE000C7CF81E090917A03911180E080937A03DF
:100AF000BECF8A8180932E028B8180932F028C81BE
:100B0000809330028D81809331028EE292E0E3CFB8
:100B10008A8180FF04C081E080930001A8CF1092F9
:100B20000001A5CF8091000180932E028EE292E019
:100B3000909335048093340411E09ACF84E893E0D5
:100B40000E94320F609388037093890380938A0315
:100B500090938B038CCF0E94260F009188031091F5
:100B6000890320918A0330918B03601B710B820BE8
:100B7000930B60932A0270932B0280932C02909324
:100B80002D028AE292E0A7CF0E94260F8B019C01E2
:100B90008D814A8150E060E070E0BA01552744271A
:100BA000582B8C81482B8B81782B80E793E00E9417
:100BB0002E165DCF0C80DD81C02D0E94260F6B01AB
:100BC0007C01CC1ADD0AE108F10880E793E00E947D
:100BD0002216AB01BC0197018601E7CF80E793E0C5
:100BE0000E946D16A1CF80E793E00E94B11690930A
:100BF00011028093100280E192E09093350480937B
:100C0000340412E035CF80E793E00E94B11660EA29
:100C100075E00E946019EBCF80E793E00E942216F6
:100C2000A8CF0E94260F6B017C0180E793E00E9411
:100C30002816C61AD70AE80AF90AC0922A02D092E0
:100C40002B02E0922C02F0922D029BCF86E292E0E2
:100C50000E94320FC0908803D0908903E0908A03ED
:100C6000F0908B036C197D098E099F0960931E0219
:100C700070931F028093200290932102809126029C
:100C800090912702A0912802B091290240918403FB
:100C9000509185036091860370918703841B950BA7
:100CA000A60BB70B8093220290932302A0932402F9
:100CB000B09325028EE192E0909335048093340442
:100CC000D7CE1A810C80DD81C02DCE010E94E9199A
:100CD000181709F4CCCE612FCE010E94F119C7CEAE
:100CE0008C819D810E94E9191FCF81E080937D0353
:100CF0008A8180937B03BBCEE091610284E0E89F10
:100D0000F0011124E55AFD4F8785968590932E02B8
:100D100080932F028EE292E070CF89E592E06DCF52
:100D20008EE00E94071063CF81E0809379039FCE0D
:100D300081E080932E0285E380932F0284E28093EA
:100D4000300210923102E1CE81E080937C038FCE9D
:100D50002F923F924F925F926F927F928F929F92CB
:100D6000AF92BF92CF92DF92EF92FF920F931F93B9
:100D7000CF93DF93CDB7DEB766970FB6F894DEBF9B
:100D80000FBECDBF8D8B9E8B1B01ED89FE8924810B
:100D90003581C9010196628173810E946019609159
:100DA000070170910801009709F407C145E0489FC9
:100DB000D001499FB00D1124AE0FBF1F429FF0011B
:100DC000439FF00D11244D895E89E40FF51F17969E
:100DD0004D915C910780F085E02D4E1B5F0B469F87
:100DE0004001479F900C569F900C1124A40160E095
:100DF00070E02101612C712CA5E0A29FF001A39F5E
:100E0000F00D11242D893E892E0F3F1F3A8B298B1F
:100E1000F901A184B12CC12CD12CA89F9001A99FCC
:100E2000300D11248D899E89820F931F9C8B8B8B93
:100E3000FC0181851F921F921F928F934D875E87C1
:100E40006F87788B7A018B0120E030E0A901C30124
:100E5000B2010E94471469837A838B839C83E9895A
:100E6000FA89A284B12CC12CD12CEB89FC89828512
:100E70001F921F921F928F93ED84FE840F85188915
:100E800020E030E0A901C301B2010E9447146D8344
:100E90007E838F839887E989FA89A384B12CC12C3A
:100EA000D12CEB89FC8983851F921F921F928F930F
:100EB000ED84FE840F85188920E030E0A901C3018C
:100EC000B2010E94471469877A878B879C87698162
:100ED0007A818B819C817727882799272091090126
:100EE0001F921F921F922F93A12CB12C6501E12C10
:100EF000F12C8701EA9420E030E0A9010E94471418
:100F0000609383036D817E818F8198857727882701
:100F10009927209109011F921F921F922F9320E081
:100F200030E0A9010E9447146093820369857A85A5
:100F30008B859C85772788279927209109011F9207
:100F40001F921F922F9320E030E0A9010E944714C6
:100F5000609381030FB6F894DEBF0FBECDBFC4010E
:100F600001972816390658F0ED89FE89848195810C
:100F70000196628173810E94601995838483C10107
:100F80000196B4010E94601966960FB6F894DEBF10
:100F90000FBECDBFDF91CF911F910F91FF90EF90CA
:100FA000DF90CF90BF90AF909F908F907F906F9089
:100FB0005F904F903F902F900895ED89FE89468174
:100FC000469F4001479F900C112410CF2F923F92D3
:100FD0004F925F926F927F928F929F92AF92BF9249
:100FE000CF92DF92EF92FF920F931F93CF93DF93F5
:100FF000CDB7DEB766970FB6F894DEBF0FBECDBF94
:101000008D8B9E8B1B01ED89FE8924813581C90161
:101010000196628173810E9460196091050170914F
:101020000601009709F407C145E0489FD001499F98
:10103000B00D1124AE0FBF1F429FF001439FF00D72
:1010400011244D895E89E40FF51F17964D915C912F
:101050000780F085E02D4E1B5F0B469F4001479FA8
:10106000900C569F900C1124A40160E070E02101C7
:10107000612C712CA5E0A29FF001A39FF00D11241B
:101080002D893E892E0F3F1F3A8B298BF901A184B0
:10109000B12CC12CD12CA89F9001A99F300D1124F7
:1010A0008D899E89820F931F9C8B8B8BFC01818580
:1010B0001F921F921F928F934D875E876F87788B49
:1010C0007A018B0120E030E0A901C301B2010E9446
:1010D000471469837A838B839C83E989FA89A28484
:1010E000B12CC12CD12CEB89FC8982851F921F92D7
:1010F0001F928F93ED84FE840F85188920E030E0E5
:10110000A901C301B2010E9447146D837E838F83BE
:101110009887E989FA89A384B12CC12CD12CEB8959
:10112000FC8983851F921F921F928F93ED84FE840A
:101130000F85188920E030E0A901C301B2010E94A7
:10114000471469877A878B879C8769817A818B812D
:101150009C81772788279927209109011F921F9248
:101160001F922F93A12CB12C6501E12CF12C87014A
:10117000EA9420E030E0A9010E94471460938003C4
:101180006D817E818F819885772788279927209187
:1011900009011F921F921F922F9320E030E0A901B6
:1011A0000E94471460937F0369857A858B859C85AF
:1011B000772788279927209109011F921F921F9254
:1011C0002F9320E030E0A9010E94471460937E0332
:1011D0000FB6F894DEBF0FBECDBFC401019728162D
:1011E000390658F0ED89FE898481958101966281E6
:1011F00073810E94601995838483C1010196B401B3
:101200000E94601966960FB6F894DEBF0FBECDBF80
:10121000DF91CF911F910F91FF90EF90DF90CF90D2
:10122000BF90AF909F908F907F906F905F904F9006
:101230003F902F900895ED89FE894681469F400199
:10124000479F900C112410CF809178038115C1F035
:1012500060E08BE00E94D31060E08AE00E94D3102F
:1012600060E089E00E94D31060E083E00E94D31028
:1012700060E085E00E94D31060E086E00C94D3101B
:101280006091830370E08BE00E94221060918203E2
:1012900070E08AE00E9422106091810370E089E092
:1012A0000E9422106091800370E083E00E9422106F
:1012B00060917F0370E085E00E94221060917E03C0
:1012C00070E086E00C942210CDB7DEB7C750D44052
:1012D0000FB6F894DEBF0FBECDBF4E0124E0821AD8
:1012E0002EEF920A8BEF91E0F4019C0111922150B4
:1012F0003040E1F7AE014F5F5F4F2A01FA019C01D8
:10130000119221503040E1F70E94CC0F80B78064E9
:1013100080BF64E670E080E090E00E94930F80B7A9
:10132000886080BF80B780728093780361E08BE033
:101330000E94991061E08AE00E94991061E089E0C2
:101340000E94991061E083E00E94991061E085E0BD
:101350000E94991061E086E00E94991060E08EE0A2
:101360000E94991062E081E10E94991062E082E19E
:101370000E94991062E083E10E94991061E088E088
:101380000E94991061E08DE00E94991060E08BE06E
:101390000E94D31060E08AE00E94D31060E089E0F0
:1013A0000E94D31060E083E00E94D31060E085E0EB
:1013B0000E94D31060E086E00E94D31060E08DE0D0
:1013C0000E94D31061E088E00E94D31026E040E044
:1013D00052EC61E070E086E993E00E94E01168E57C
:1013E00071E086E993E00E9413138BE592E00E947E
:1013F000CF0290935A028093590260E773E08BE525
:1014000092E00E94BD03F82E4091590250915A0279
:1014100034E0839F80011124055A1D4FF40111828D
:101420001082B401F80186850E941A02F4017080CE
:1014300061804091590250915A021A821982B20178
:10144000F80187850E941A0249805A80709207012C
:1014500060920801509206014092050181E080935C
:101460004202109245026CE671E086E993E00E9428
:1014700006138091420267E471E0811102C06FE4BB
:1014800071E086E993E00E9413138FEF9FEF909332
:1014900036028093350210923402109233020E9479
:1014A0004519549A8FEF90E0E7EBFBE03197F1F7A5
:1014B00000C000000197C1F754987894C750DC4FE2
:1014C00019821882C95FD340C950DC4F1982188233
:1014D000C75FD340CD5FDB4F1882C350D440312C5F
:1014E000C150DC4F188219821A821B82CF5FD34011
:1014F000A12CB12C650122E3822E912C0E9461184F
:1015000080917A038111FACF8091790381110E9431
:1015100010050E94260FC550DC4F6883CB5FD34077
:10152000C450DC4F7883CC5FD340C350DC4F8883FA
:10153000CD5FD340C250DC4F9883CE5FD340C550BF
:10154000DC4F488159816A817B81CB5FD34080E742
:1015500093E00E94A0140E944F0FC150DC4F2881DD
:1015600039814A815B81CF5FD340621B730B840B4F
:10157000950B603D774081059105D0F087E392E0BF
:101580000E947F170E944F0FC150DC4F6883CF5FCE
:10159000D340C050DC4F7883C050D440CF5FDB4F86
:1015A0008883C150D440CE5FDB4F9883C250D44073
:1015B00087E392E00E941517919581959109909388
:1015C00034028093330287E392E00E944A178093AB
:1015D0003202843009F41AC18330A1F4CD5FDB4FAD
:1015E0004881C350D440411107C081E0909100016F
:1015F000911180E08093000151E0CD5FDB4F588373
:10160000C350D44080910001811509F405C1809137
:101610007803811101C18091330290913402892BAA
:1016200081F06DE771E086E993E00E940613609116
:101630003302709134024AE050E086E993E00E9460
:10164000DD13809132028115B1F062E971E086E923
:1016500093E00E9406134AE050E06091320286E96E
:1016600093E00E94191480913202853021F4339462
:10167000832D8170382E80917C03811509F445C03B
:1016800010927C038BE592E00E94CF0290935A0265
:101690008093590260E773E08BE592E00E94BD03FE
:1016A000F82E4091590250915A0294E0899F80018E
:1016B0001124055A1D4FC450DE4F7882CC5FD140B3
:1016C000C350DE4F6882CD5FD140BE0164507E4F73
:1016D000F80186850E941A02C450DE4F7880CC5FE4
:1016E000D140C350DE4F6880CD5FD1404091590258
:1016F00050915A025A824982BE016F5F7F4FF801B2
:1017000087850E941A0249805A8080917D03811545
:1017100081F110927D034091590250915A02C450B8
:10172000DE4F7882CC5FD140C350DE4F6882CD5F00
:10173000D140BE0164507E4F80917B030E941A020B
:10174000C450DE4F7880CC5FD140C350DE4F6880FC
:10175000CD5FD1404091590250915A025A8249823C
:10176000BE016F5F7F4F80917B030E941A02498008
:101770005A80809133029091340297FFF6C1311064
:10178000B5C16BE971E086E993E00E9406136091B0
:101790000701709108014AE050E086E993E00E9459
:1017A00033146BEA71E086E993E00E9406134091DE
:1017B000330250913402052E000C660B770B80919A
:1017C000070190910801480F591F611D711D2AE002
:1017D00030E086E993E00E94F1138090330290900C
:1017E00034028091070190910801A401092C000C9A
:1017F000660B770B480F591F611D711D4230510553
:101800006105710574F1880E991E2EC0CD5FDB4F06
:101810001882C350D440F6CE80917803811123C240
:1018200060E070E08BE00E94221060E070E08AE0EF
:101830000E94221060E070E089E00E94221060E0C7
:1018400070E083E00E94221060E070E085E00E947A
:10185000221060E070E086E00E9422100E94260FB5
:101860004DCE88248394912C6FEB71E086E993E050
:101870000E9406134AE050E0B40186E993E00E941A
:101880003314409101015091020160910301709164
:101890000401C550DC4F88819981AA81BB81CB5F4F
:1018A000D3408A199B09AC09BD0984179507A6077F
:1018B000B70708F423CE60E773E08BE592E00E945F
:1018C000BD03282EF81609F44AC0409159025091E0
:1018D0005A02F4E08F9F80011124055A1D4FC45015
:1018E000DE4F7882CC5FD140C350DE4F6882CD5F3F
:1018F000D140BE0164507E4FF80186850E941A02D5
:10190000C450DE4F7880CC5FD140C350DE4F68803A
:10191000CD5FD1404091590250915A025A8249827A
:10192000BE016F5F7F4FF80187850E941A024980D0
:101930005A8070920701609208015092060140920D
:101940000501872C962CC750DC4F19821882C95F7D
:10195000D340C950DC4F19821882C75FD340E09052
:101960000701F0900801E814F904B1F100E010E07B
:10197000C950DC4F28813981C75FD340B90180E06D
:1019800090E094011F921F923F938F92A12CB12C53
:10199000650120E030E0A9010E944714CC5FDB4FD5
:1019A0006883C450D440CB5FDB4F7883C550D440AC
:1019B000CC5FDB4F48815981C450D440C950DC4FC3
:1019C00059834883C75FD3409092080180920701F2
:1019D0000F900F900F900F90C450DE4F7882CC5F25
:1019E000D140C350DE4F6882CD5FD140C950DC4F3B
:1019F00068817981C75FD340CE0184509E4F0E9499
:101A0000A806C950DC4F8883C75FD340C850DC4F5D
:101A10009883C85FD340C450DE4F7880CC5FD140FC
:101A2000C350DE4F6880CD5FD140E0900501F0905B
:101A30000601E814F904B1F100E010E0C750DC4FF2
:101A4000E881F981C95FD340BF0180E090E0940153
:101A50001F921F923F938F92A12CB12C650120E021
:101A600030E0A9010E944714CA5FDB4F6883C6506B
:101A7000D440C95FDB4F7883C750D440CA5FDB4F87
:101A800028813981C650D440C750DC4F3983288320
:101A9000C95FD34090920601809205010F900F908C
:101AA0000F900F905A824982C750DC4F688179812C
:101AB000C95FD340CE0101960E94E607C750DC4FB4
:101AC0008883C95FD340C650DC4F9883CA5FD34038
:101AD00049805A800E942409F22CC550DC4FA8800E
:101AE000B980CA80DB80CB5FD34008CD6FEC71E05A
:101AF00086E993E00E9406134AE050E060910901F4
:101B000086E993E00E9419146CED71E086E993E098
:101B10000E94061380910901609133027091340292
:101B2000680F711D4AE050E086E993E00E94DD13E2
:101B3000209109018091330290913402820F911D0E
:101B400097FF02C080E090E08093090160EF71E0B0
:101B500086E993E00E9406134AE050E06091090193
:101B600086E993E00E9419148CCE892B09F489CE62
:101B7000311047C06BE971E086E993E00E940613DB
:101B800060910701709108014AE050E086E993E016
:101B90000E9433146BEA71E086E993E00E94061319
:101BA0004091330250913402052E000C660B770BE6
:101BB0008091070190910801480F591F611D711D07
:101BC0002AE030E086E993E00E94F113809033022E
:101BD000909034028091070190910801A401092C92
:101BE000000C660B770B480F591F611D711D4336A2
:101BF0005105610571050CF406CE84E6882E912C02
:101C000033CE6FEC71E086E993E00E9406134AE060
:101C100050E06091090186E993E00E9419146CED8F
:101C200071E086E993E00E940613809109016091BA
:101C3000330270913402680F711D4AE050E086E96A
:101C400093E00E94DD1380910901209133023091CD
:101C50003402A901480F511D820F4E3F51050CF46B
:101C600073CF8FEF71CF83B7817F83BF83B78160DD
:101C700083BF889583B78E7F83BF40CC1F920F921E
:101C80000FB60F9211242F933F934F935F936F934F
:101C90007F938F939F93AF93BF93EF93FF9300B680
:101CA00005FC13C010927803FF91EF91BF91AF91A3
:101CB0009F918F917F916F915F914F913F912F9164
:101CC0000F900FBE0F901F90189581E080937803BE
:101CD00060E08BE00E94D31060E08AE00E94D310A5
:101CE00060E089E00E94D31060E083E00E94D3109E
:101CF00060E085E00E94D31060E086E00E94D3108F
:101D0000D3CFEF920F93CF93DF9380E793E00E94BE
:101D1000961410925C0210925B0210925E02109276
:101D20005D0210925F0210926002109261021092A6
:101D30006202109264021092630210926602109284
:101D40006502E7E6F2E08CE8DF011D928A95E9F78B
:101D5000E3EFF2E084E11082118212821382DF014C
:101D60001596ED01982F19929A95E9F77996A3E0C7
:101D7000E037FA0781F7E12C04E023E142E161E179
:101D800087E392E00E94B816DF91CF910F91EF9018
:101D9000089578944F934FB74F935F936F937F93CA
:101DA0008F939F9340918E0350918F036091900386
:101DB0007091910380918D0390918C039F5F93307C
:101DC00080F5835D8D3780F54F5F5F4F6F4F7F4F9D
:101DD00080938D0340938E0350938F036093900301
:101DE00070939103409192035091930360919403F7
:101DF000709195034F5F5F4F6F4F7F4F40939203FA
:101E000050939303609394037093950390938C0382
:101E10009F918F917F916F915F914F914FBF4F91A4
:101E20001895815D90E0CECF8D574E5F5F4F6F4F1D
:101E30007F4FCECF2FB7F8946091920370919303A8
:101E400080919403909195032FBF08952FB7F89434
:101E500060918E0370918F03809190039091910314
:101E60002FBF08950F931F93FC014FB7F894609113
:101E70008E0370918F038091900390919103009154
:101E800092031091930320919403309195034FBFD7
:101E900000831183228333831F910F9108958F92C2
:101EA0009F92AF92BF92CF92DF92EF92FF923FB795
:101EB000F8948091920390919303A0919403B09130
:101EC000950326B5A89B05C02F3F19F00196A11DCB
:101ED000B11D3FBFBA2FA92F982F88276C017D0114
:101EE000C20ED11CE11CF11CA5E0B0E0A7019601D7
:101EF0000E94CF194B015C01C701B60123E030E01D
:101F000040E050E00E948819C501B401620F731FC0
:101F1000841F951FFF90EF90DF90CF90BF90AF9000
:101F20009F908F9008958F929F92AF92BF92CF9281
:101F3000DF92EF92FF926B017C010E944F0F4B01E9
:101F40005C01C114D104E104F104E9F00E944C19D0
:101F50000E944F0F681979098A099B09683E7340EE
:101F60008105910570F321E0C21AD108E108F1085A
:101F700088EE880E83E0981EA11CB11CC114D10408
:101F8000E104F10429F7FF90EF90DF90CF90BF902C
:101F9000AF909F908F900895789484B5826084BDAF
:101FA00084B5816084BD85B5826085BD85B581605D
:101FB00085BDEEE6F0E0808181608083E1E8F0E0BD
:101FC0001082808182608083808181608083E0E8EC
:101FD000F0E0808181608083E1EBF0E080818460CB
:101FE0008083E0EBF0E0808181608083EAE7F0E0CD
:101FF00080818460808380818260808380818E7F05
:1020000080838081806880831092C10008958E3023
:1020100008F08E5090910A019295990F990F907C3B
:102020008770892B80937C0080917A0080648093F4
:102030007A0080917A0086FDFCCF809178009091A3
:10204000790008959B016115710519F460E00C9405
:10205000D3106F3F710511F461E0F9CFE82FF0E084
:10206000E859FF4FE491E43059F150F4E230C9F0FF
:10207000E330E1F0E13081F0203831053CF3ECCF82
:10208000E73041F1E830C1F78091B0008062809381
:10209000B0006093B400089584B5806884BD67BDC6
:1020A000089584B5806284BD68BD089580918000E4
:1020B0008068809380007093890060938800089501
:1020C0008091800080628093800070938B00609389
:1020D0008A0008958091B00080688093B00060937A
:1020E000B3000895843081F050F48230A9F0833039
:1020F00079F4809180008F778093800008958730F5
:1021000071F0883091F00895809180008F7DF4CF38
:1021100084B58F7784BD089584B58F7DFBCF809182
:10212000B0008F778093B00008958091B0008F7DCC
:10213000F9CFCF93DF9390E0FC01E458FF4F249157
:1021400080579F4FFC0184918115C9F090E0880F62
:10215000991FFC01E854FF4FA591B591FC01E25590
:10216000FF4FC591D5919FB761110CC0F8948C9128
:10217000209582238C938881282328839FBFDF9119
:10218000CF910895623051F4F8943C91822F80955C
:1021900083238C938881822B8883F0CFF8948C9151
:1021A000822B8C93EBCF1F93CF93DF93162F282F87
:1021B00030E0F901E859FF4F8491F901E458FF4FED
:1021C000D491F901E057FF4FC491C115A1F08111DD
:1021D0000E947210EC2FF0E0EE0FFF1FE255FF4F50
:1021E000A591B5919FB7F8948C91111108C0D09525
:1021F000D823DC939FBFDF91CF911F9108958D2B42
:102200008C93F8CFCF93DF93282F30E0F901E85972
:10221000FF4F8491F901E458FF4FD491F901E05741
:10222000FF4FC491C11581F081110E947210EC2FF3
:10223000F0E0EE0FFF1FEC55FF4FA591B591EC912B
:10224000ED2381E0E11101C080E090E0DF91CF91CA
:102250000895FC01818D228D90E0805C9F4F821B50
:1022600091098F7399270895FC01918D828D98179C
:1022700031F0828DE80FF11D858D90E008958FEF8C
:102280009FEF0895FC01918D828D981761F0A28DCA
:10229000AE0FBF2FB11D5D968C91928D9F5F9F7386
:1022A000928F90E008958FEF9FEF0895FC01A48D29
:1022B000A80FB92FB11DA35ABF4F2C91848D90E068
:1022C00001968F739927848FA689B7892C93A0894B
:1022D000B1898C9180648C93938D848D981306C002
:1022E0000288F389E02D80818F7D80830895CF93CC
:1022F000DF93EC01888D811111C0DF91CF9108959A
:102300000FB607FC0DC0808185FF0AC0A889B98976
:102310008C9185FF05C0CE010E945611EA89FB8988
:10232000808185FDEDCFA889B9898C9186FFE8CFA2
:10233000E4CFEF92FF920F931F93CF93DF93EC01C3
:10234000F62E81E0888F9B8D8C8D981316C0E889BE
:10235000F989808185FF11C0EE89FF896083E88952
:10236000F98980818064808381E090E0DF91CF9162
:102370001F910F91FF90EF9008950B8D10E00F5F6C
:102380001F4F0F731127E02E8C8D8E1569F0EB8D8A
:10239000EC0FFD2FF11DE35AFF4FF0820B8FEA89FE
:1023A000FB8980818062DFCF0FB607FCEDCFE88923
:1023B000F989808185FFE8CFCE010E945611E4CFD4
:1023C000DF92EF92FF920F931F93CF93DF93EC0175
:1023D000D42EE52EF62E072F122F60EC76EC8DE230
:1023E00090E0242F352F4F2D502F0E948819215017
:1023F0003109410951095695479537952795E8893F
:10240000F98982E08083211580E13807A8F0E88906
:10241000F989108260E673EE86E190E02D2D3E2D65
:102420004F2D502F0E94881921503109410951091F
:102430005695479537952795EC85FD853083EE8534
:10244000FF852083188EEC89FD891083EA89FB893A
:10245000808180618083EA89FB89808188608083B4
:10246000EA89FB89808180688083EA89FB89808191
:102470008F7D8083DF91CF911F910F91FF90EF901F
:10248000DF9008952F932FB72F938F939F93EF9300
:10249000FF93E091A603F091A7038081E091AC0344
:1024A000F091AD0382FD19C090818091AF038F5FE1
:1024B0008F732091B003821741F0E091AF03F0E0F9
:1024C000EA56FC4F958F8093AF03FF91EF919F9158
:1024D0008F912F912FBF2F9118958081F6CF1F924A
:1024E0000F920FB60F9211242F933F934F935F9348
:1024F0006F937F938F939F93AF93BF93EF93FF93CC
:1025000086E993E00E945611FF91EF91BF91AF9140
:102510009F918F917F916F915F914F913F912F91FB
:102520000F900FBE0F901F901895E6E9F3E013820D
:10253000128288EE93E0A0E0B0E084839583A683C6
:10254000B78384E092E09183808385EC90E0958767
:10255000848784EC90E09787868780EC90E0918B6D
:10256000808B81EC90E0938B828B82EC90E0958B5A
:10257000848B86EC90E0978B868B118E128E138E57
:10258000148E0895CF92DF92EF92FF920F931F93D4
:10259000CF93DF937C016A0100E010E00C151D056C
:1025A00051F4C801DF91CF911F910F91FF90EF90EF
:1025B000DF90CF900895EB01D701ED91FC91019050
:1025C000F081E02D6991C7010995892B51F30F5FC7
:1025D0001F4FBE01E3CFCF93DF93EC01DB01AB2BA9
:1025E00081F0FB0101900020E9F73197AF01461B14
:1025F000570BE881F9810280F381E02DDF91CF91C3
:10260000099480E090E0DF91CF9108950C94EB1253
:10261000DC01ED91FC910190F081E02D09946DEFCA
:1026200071E00C94EB120F931F93CF93DF93D82F8D
:10263000C92F0E94EB128C018D2F9C2F0E940F132B
:10264000800F911FDF91CF911F910F9108952F92CD
:102650003F924F925F926F927F928F929F92AF9232
:10266000BF92CF92DF92EF92FF920F931F93CF937F
:10267000DF93CDB7DEB7A1970FB6F894DEBF0FBEDC
:10268000CDBF1C01142F052FB62EA72E19A2223064
:1026900008F42AE04E0181E2880E911CC22ED12C52
:1026A000E12CF12C612F702F8B2D9A2DA701960113
:1026B0000E948819412E502E6B2C7A2C122F032F3A
:1026C000B42EA52E6A3034F5605DF40162934F019B
:1026D0004C145D046E047F0428F7BF01C1010E9401
:1026E000EB12A1960FB6F894DEBF0FBECDBFDF91FF
:1026F000CF911F910F91FF90EF90DF90CF90BF90FF
:10270000AF909F908F907F906F905F904F903F9091
:102710002F900895695CD9CFCF92DF92EF92FF920C
:102720000F931F93CF93DF93EC016A017B01F901B3
:10273000EF2B79F4E881F9810190F081E02D642F8D
:10274000DF91CF911F910F91FF90EF90DF90CF908D
:1027500009942A303105E9F42AE0F7FE1AC06DE247
:102760000E9408138C0144275527BA014C195D09B2
:102770006E097F092AE0CE010E942713800F911F66
:10278000DF91CF911F910F91FF90EF90DF90CF904D
:102790000895B701A601CE01DF91CF911F910F914E
:1027A000FF90EF90DF90CF900C9427139A01AB012C
:1027B000770F660B770B0C948C130F931F93CF93AB
:1027C000DF93D82FC92F0E94D6138C018D2F9C2FF9
:1027D0000E940F13800F911FDF91CF911F910F91D6
:1027E00008950F931F93CF93DF93D82FC92F0E9483
:1027F0008C138C018D2F9C2F0E940F13800F911F23
:10280000DF91CF911F910F910895DC01F901EF2B1A
:1028100039F4ED91FC910190F081E02D642F099441
:102820000C9427139A01462F50E060E070E00C945E
:1028300005140F931F93CF93DF93D82FC92F0E94B6
:1028400012148C018D2F9C2F0E940F13800F911F4B
:10285000DF91CF911F910F9108959A01AB0160E034
:1028600070E00C9405140F931F93CF93DF93D82F30
:10287000C92F0E942D148C018D2F9C2F0E940F13A5
:10288000800F911FDF91CF911F910F9108954F926B
:102890005F926F927F92AF92BF92CF92DF92EF9250
:1028A000FF920F931F93CF93DF9300D000D0CDB74B
:1028B000DEB729013A01A982BA82CB82DC829B0170
:1028C000AC0124193509460957098D899E89AF89BC
:1028D000B88DBC01CD01A980BA80CB80DC806A199B
:1028E0007B098C099D090E945019A80197012419A0
:1028F0003509460957090E94AA19C601B501620F98
:10290000731F841F951F0F900F900F900F90DF91F2
:10291000CF911F910F91FF90EF90DF90CF90BF90DC
:10292000AF907F906F905F904F900895FC01108260
:1029300011821282138214821582168217820895E0
:102940004F925F926F927F928F929F92AF92BF92BF
:10295000CF92DF92EF92FF92CF93DF93EC016A0167
:102960007B018C819D81AE81BF81A7019601281BCF
:10297000390B4A0B5B0BCA01B90160363AEE73079B
:102980008105910520F188809980AA80BB8020E68E
:102990003AEE40E050E00E9488192B013C01CA0148
:1029A000B901680D791D8A1D9B1D20EA33E24AE8B2
:1029B0005CE00E948819688379838A839B83C418AA
:1029C000D508E608F708CC82DD82EE82FF826881B6
:1029D00079818A819B81DF91CF91FF90EF90DF9089
:1029E000CF90BF90AF909F908F907F906F905F90AF
:1029F0004F900895CF92DF92EF92FF920F931F9323
:102A0000CF93DF938A01D62FC72FBA018D2F9C2F2A
:102A100020E837E842E253E00E94881969017A0110
:102A2000B8018D2F9C2F20EA35E040E050E00E9455
:102A30008819C20ED31EE41EF51EB8018D2F9C2FDF
:102A400020E834E140E250E00E948819C21AD30A1B
:102A5000E40AF50AB8018D2F9C2F20E03EE14AE8F8
:102A60005CE00E948819C701B601621B730B840BDE
:102A7000950B2DE631E040E050E00E948819C90135
:102A8000DF91CF911F910F91FF90EF90DF90CF904A
:102A90000895EF92FF920F931F93CF93DF937A01E4
:102AA0008B010E94FA14EC01B701C80120EA35E05D
:102AB00040E050E00E94881989019A01CE0164E645
:102AC00070E00E946019CB01800F911F4DE651E02C
:102AD000C49F9001C59F300DD49F300D1124821BDF
:102AE000930BD695C795D695C7958C1B9D0BDF91FB
:102AF000CF911F910F91FF90EF9008950E9449157B
:102B000045E0489F9001499F300D1124C90102966C
:102B100069E970E00E94601983E06A3008F087EF8D
:102B2000860F0895CF93DF930E944915EC01282F5B
:102B30002F5F35E03C9FC0013D9F900D1124029610
:102B400069E970E00E94601939E9639FC0011124AE
:102B5000029665E070E00E947419822F861BDF9157
:102B6000CF9108957F928F929F92AF92BF92CF9212
:102B7000DF92EF92FF920F931F93CF93DF93D82EA4
:102B8000E92EF42E052F162FD72F0E947E15C82F61
:102B90008DEF8C0F8930B8F58CEF8C0F873008F4EF
:102BA0004FC06F2D702F812F9D2F20EA35E040E020
:102BB00050E00E9488194B015C01CA01B9016D5FA8
:102BC0007F4F8F4F9F4F27E030E040E050E00E9462
:102BD0008819762E4F2D502F612F7D2F8D2D9E2DF4
:102BE0000E949215982F9719C33079F498305CF0B1
:102BF000711026C088E788169104A104B10400F57D
:102C000081E09F307CF480E00DC01916CCF4983040
:102C1000D4F77110F8CF81E09CE389169104A104E8
:102C2000B10488F7DF91CF911F910F91FF90EF9042
:102C3000DF90CF90BF90AF909F908F907F9008953E
:102C400081E0F0CFFC0160817181828193810895E0
:102C5000FC01648175818681978108950F931F938C
:102C6000FC0140835183628373830483158326832D
:102C700037831F910F910895CF92DF92EF92FF92C9
:102C80006A017B01B701A6010E94B215682F70E0AE
:102C90007195619571096C737727A7019601260FCD
:102CA000371F411D511DCA01B90120EA35E040E03E
:102CB00050E00E948819CA01B9016D5F7F4F8F4FA4
:102CC0009F4F27E030E040E050E00E948819862FB7
:102CD000FF90EF90DF90CF900895FC0140815181EB
:102CE000628173810C943C16CF92DF92EF92FF9237
:102CF0001F93CF93DF93D82FC92F6A017B01B701B0
:102D0000A6010E943C16182FB701A6018D2F9C2FFB
:102D10000E94B215682F70E07195619571096C730E
:102D20007727A7019601260F371F411D511DCA01A4
:102D3000B90120EA35E040E050E00E94881920EA1D
:102D400035E0129FA001139F500D1124CA01860F78
:102D5000971FDF91CF911F91FF90EF90DF90CF9061
:102D60000895FC0140815181628173810C94741635
:102D7000EF920F93CF93DF93EC01862F6883498303
:102D80002A83EB821D821C821F821E8208871A867C
:102D9000198691E09B871D861C869E879F87188ACF
:102DA000198A1B8A1A8A1D8A1C8A28EE33E03F8BF7
:102DB0002E8B20E931E0398F288F1A8E1B8E1C8EC6
:102DC0001D8E1F8E1E8E19A218A2E926EE0C67FD1D
:102DD00003C06E2D0E949910898187FD03C06E2D5E
:102DE0000E9499108A8187FD03C06E2D0E94991060
:102DF00088810E9402112B812817190621F483E093
:102E000090E09F838E8389810E9402112B81281775
:102E1000190631F48E819F8121E082279F838E8362
:102E2000DF91CF910F91EF900895FC0184819581FE
:102E30002085223001F5282F217033273583248304
:102E40002085243021F49595879595958795208543
:102E5000223011F495958795238540E0211519F0CE
:102E600021853285432F242F30E097FF0EC0C90102
:102E70008095909508952085243021F49C0123703D
:102E80003327DCCF15821482DBCF009711F0C90104
:102E900001960895FC018485958524853585233028
:102EA000310521F0009711F0158614860895EF92F0
:102EB000FF920F931F93CF938C01FC01C1898281F4
:102EC000C11589F00E9407107C01F801868D978D4D
:102ED000E816F9066CF0C1E080A191A18E159F055E
:102EE0003CF0C0E005C00E940211C1E0892BC9F38B
:102EF0008C2FCF911F910F91FF90EF900895CF925B
:102F0000DF92EF92FF921F93CF93DF93EC018881C2
:102F100087FD46C0998197FD43C09B85911561F05F
:102F200029853A85265031093A87298729853A85A6
:102F300037FF02C01A8619860E9402112B8110E009
:102F40002817190609F413E089810E9402112B81C8
:102F50002817190611F481E018278E819F81811BA3
:102F600080FF59C0212F110F330B3F832E832C81FB
:102F70003D8182708150990B280F391F3D832C832E
:102F800081E09B85911561F0811551F089859A85C5
:102F90008F3C9B4028F489859A85C2969A878987B9
:102FA0000E94260F6B017C018A8D9B8DAC8DBD8D9F
:102FB000C816D906EA06FB0620F41A8E1B8E1C8E54
:102FC0001D8E8A81181634F0811148C088898115B8
:102FD00009F444C08A8D9B8DAC8DBD8DA7019601EF
:102FE000281B390B4A0B5B0B2A3031054105510573
:102FF000A8F1CA8EDB8EEC8EFD8ECE010E94571793
:103000002A893B899B81981741F02230310570F560
:103010001B8A1A8A16C080E0B4CF2F5F3F4F3B8BCC
:103020002A8B8E899F896AE070E00E94601962177E
:10303000730738F48F85811521F083E090E09D8738
:103040008C878C899D89009749F001979D8B8C8B8B
:10305000892B21F485E090E09D878C87DF91CF91CB
:103060001F91FF90EF90DF90CF9008958C859D8504
:10307000039739F484E090E09D878C871D8A1C8A31
:10308000C7CF2C893D892230310568F0888D998D14
:103090006AE070E00E9460192617370708F0B8CF81
:1030A00086E090E0E9CF8E8561E070E0811531F037
:1030B000888D998D6AE070E00E9460196C8B7D8B21
:1030C000A7CFCF93DF9380914304835087FD29C01E
:1030D000909141049D3219F5883009F5809147049B
:1030E000CCE0D0E0C81BD109C85BDB4F83EC8093F8
:1030F00036048AE580930C0110923304888180762F
:10310000811509F45FC0CE010E941B059F819111BA
:1031100004C09E81981708F4892F80930B011092A8
:10312000430480910C0184FF3FC080910B018F3FCD
:10313000D9F1C82F893008F0C8E0982F9C1B9093D4
:103140000B019091360428E892279093360481155C
:10315000E9F080913404909135042091330426FFE6
:1031600088C0FC012C2F47E354E03491DA013C93F2
:103170004F5F5F4F31962A95C1F701962FEF2C0FC5
:10318000820F911D90933504809334046C2F87E354
:1031900094E00E94D60084E08C0FC83019F09FEFB5
:1031A00090930B0180930C0184E199B1947191117A
:1031B00006C08A95D1F71092450410924604DF911B
:1031C000CF9108952A8110923F04998191110AC0EC
:1031D000109240042FE334E082E0309335042093D2
:1031E000340494CF953029F4209345042FE334E040
:1031F000F4CF963071F59B81913059F484ED90E0D5
:10320000909335048093340482E190E490933304E6
:103210007DCF923019F482EC90E0F2CF9330A9F791
:10322000211108C08EE091E090933504809334041E
:1032300084E0EBCF213019F48CEF90E0E1CF223025
:1032400021F786EE90E0909335048093340486E174
:10325000DCCF983051F0993019F420934404C6CF54
:1032600081E09A3019F280E0C1CF24E434E081E0BB
:10327000B4CFDC012C2F47E354E0FA013D913083B9
:103280004F5F5F4F2A95C9F778CFE9E6F0E080817C
:1032900082608083E89A08950895F8940C94FF1949
:1032A000DB018F939F930E94CF19BF91AF91A29F93
:1032B000800D911DA39F900DB29F900D1124089534
:1032C000AA1BBB1B51E107C0AA1FBB1FA617B7074C
:1032D00010F0A61BB70B881F991F5A95A9F7809568
:1032E0009095BC01CD01089597FB072E16F400942C
:1032F00007D077FD09D00E94601907FC05D03EF485
:10330000909581959F4F0895709561957F4F089591
:10331000A1E21A2EAA1BBB1BFD010DC0AA1FBB1FD9
:10332000EE1FFF1FA217B307E407F50720F0A21B4B
:10333000B30BE40BF50B661F771F881F991F1A94B8
:1033400069F760957095809590959B01AC01BD01E2
:10335000CF010895052E97FB1EF400940E94C11919
:1033600057FD07D00E94881907FC03D04EF40C9437
:10337000C11950954095309521953F4F4F4F5F4F64
:10338000089590958095709561957F4F8F4F9F4FD1
:103390000895EE0FFF1F0590F491E02D09940E940F
:1033A000DA19A59F900DB49F900DA49F800D911DDB
:1033B00011240895A29FB001B39FC001A39F700D77
:1033C000811D1124911DB29F700D811D1124911D2D
:1033D0000895F999FECF92BD81BDF89A992780B5DD
:1033E0000895262FF999FECF1FBA92BD81BD20BD49
:1033F0000FB6F894FA9AF99A0FBE01960895F894C8
:10340000FFCF7905880592059E05AB05610670061C
:10341000750626062D0542054D0571059006940694
:10342000C405DA05EE05F3050C0611067C068D06CB
:0634300003069806A40645
:10343600010A00000032003200FF01FF5A456E7497
:10344600657265642072656164206379636C6520CA
:1034560066726F6D20454550524F4D00417474653C
:103466006D7074696E6720746F2072656164206385
:1034760079636C653A2000656E61626C6564006410
:10348600697361626C6564004C616D70207365726E
:1034960069616C206163746976652E0041636365BA
:1034A6006C65726174696F6E2069732000456E6386
:1034B6006F646572206368616E6765642062793A3D
:1034C6002000427574746F6E3A20004F6C6420665B
:1034D60072616D65446973743A200064656C746149
:1034E600202B206672616D65446973743A20006E04
:1034F6006577206672616D65446973743A20004F82
:103506006C64206272696768743A200064656C7442
:1035160061202B206375724272696768743A2000D5
:103526006E6577206272696768743A20000D0A003A
:10353600000000009911C2122911421134117711AD
:00000001FF
